:0200000480007A
:10000000971700009387070073100034F3E0003463
:10001000F31000347361003473110034F3E10F34D2
:10002000F31100347362083473120034F3E20734BE
:10003000F312003423A0070023A2170023A42700F3
:1000400023A6370023A8470023AA570097120000D1
:100050009382C2FC73100034F3E5003473660034FD
:10006000F3E60F3473670834F3E70734736800343A
:1000700023A0020023A2B20023A4C20023A6D20020
:1000800023A8E20023AAF20023AC0201971000008B
:10009000938080FA375A1632130A8A4973100A3449
:1000A00073E00734F31A0A3423A0000023A250019E
:1000B00023A44001171500001305C5F4971500008F
:1000C000938545F8370610F01306C6F26306B502AD
:1000D0008326C5002320D600832685002320D60052
:1000E000832645002320D600832605002320D60042
:1000F000130505016FF09FFD370510F0130505F29C
:0401000023200500B3
:10100000FFFFFFFFFFFFFFFFFFFFFFFFFFFFFFFFF0
:10101000FFFFFFFFFFFFFFFFFFFFFFFFFFFFFFFFE0
:10102000FFFFFFFFFFFFFFFFFFFFFFFFFFFFFFFFD0
:10103000FFFFFFFFFFFFFFFFFFFFFFFFFFFFFFFFC0
:040000058000000077
:00000001FF
